 vcom_proxy

 Timestamp is 4b812afa (Sun Feb 21 21:45:46 2010)

 Preferred load address is 10000000

 Start         Length     Name                   Class
 0001:00000000 00008704H .text                   CODE
 0001:00008710 000000f6H .text$x                 CODE
 0001:00008810 0000002dH .text$yd                CODE
 0002:00000000 00000114H .idata$5                DATA
 0002:00000114 00000004H .CRT$XCA                DATA
 0002:00000118 00000004H .CRT$XCZ                DATA
 0002:0000011c 00000004H .CRT$XIA                DATA
 0002:00000120 0000000cH .CRT$XIC                DATA
 0002:0000012c 00000004H .CRT$XIZ                DATA
 0002:00000130 00000004H .CRT$XPA                DATA
 0002:00000134 00000004H .CRT$XPZ                DATA
 0002:00000138 00000004H .CRT$XTA                DATA
 0002:0000013c 00000004H .CRT$XTZ                DATA
 0002:00000140 00001a50H .rdata                  DATA
 0002:00001b90 000000dcH .rdata$r                DATA
 0002:00001c70 00000028H .rdata$sxdata           DATA
 0002:00001c98 00000004H .rtc$IAA                DATA
 0002:00001c9c 00000004H .rtc$IZZ                DATA
 0002:00001ca0 00000004H .rtc$TAA                DATA
 0002:00001ca4 00000004H .rtc$TZZ                DATA
 0002:00001ca8 00000508H .xdata$x                DATA
 0002:000021b0 00000000H ATL$__a                 DATA
 0002:000021b0 00000000H ATL$__z                 DATA
 0002:000021b0 00000050H .idata$2                DATA
 0002:00002200 00000014H .idata$3                DATA
 0002:00002214 00000114H .idata$4                DATA
 0002:00002328 000004e8H .idata$6                DATA
 0002:00002810 000000dbH .edata                  DATA
 0003:00000000 00000cb4H .data                   DATA
 0003:00000cc0 00000bfcH .bss                    DATA

  Address         Publics by Value              Rva+Base       Lib:Object

 0000:00000000       __except_list              00000000     <absolute>
 0000:0000000a       ___safe_se_handler_count   0000000a     <absolute>
 0000:00000000       ___ImageBase               10000000     <linker-defined>
 0001:00000000       _DllMain@12                10001000 f   dllmain.obj
 0001:00000010       _SPGetOpenFileName         10001010 f   vcom_proxy.obj
 0001:00000070       _SPGetSaveFileName         10001070 f   vcom_proxy.obj
 0001:000000d0       ?InvokeNewDialog@SPVistaCOMProxy@@QAEHW4_NEW_FILE_DIALOG_INVOKE_TYPE@@PAUtagOFNW@@PBU_GUID@@@Z 100010d0 f   vcom_proxy.obj
 0001:000005d0       ??1?$CComPtr@UIObjectCollection@@@ATL@@QAE@XZ 100015d0 f i vcom_proxy.obj
 0001:000005d0       ??1?$CComPtr@UIShellLinkW@@@ATL@@QAE@XZ 100015d0 f i vcom_proxy.obj
 0001:000005d0       ??1?$CComQIPtr@UIObjectArray@@$1?_GUID_92ca9dcd_5622_4bba_a805_5e9f541bd8c9@@3U__s_GUID@@B@ATL@@QAE@XZ 100015d0 f i vcom_proxy.obj
 0001:000005d0       ??1?$CComPtr@UIObjectArray@@@ATL@@QAE@XZ 100015d0 f i vcom_proxy.obj
 0001:000005d0       ??1?$CComPtr@UIFileSaveDialog@@@ATL@@QAE@XZ 100015d0 f i vcom_proxy.obj
 0001:000005d0       ??1?$CComPtr@UICustomDestinationList@@@ATL@@QAE@XZ 100015d0 f i vcom_proxy.obj
 0001:000005d0       ??1?$CComQIPtr@UIPropertyStore@@$1?_GUID_886d8eeb_8cf2_4446_8d02_cdba1dbdcf99@@3U__s_GUID@@B@ATL@@QAE@XZ 100015d0 f i vcom_proxy.obj
 0001:000005d0       ??1?$CComPtr@UIFileOpenDialog@@@ATL@@QAE@XZ 100015d0 f i vcom_proxy.obj
 0001:000005e0       _CreateJumpList            100015e0 f   vcom_proxy.obj
 0001:00000640       _CreateJumpListTask        10001640 f   vcom_proxy.obj
 0001:000006a0       ?CreateJumpList@SPVistaCOMProxy@@QAEHPB_W00@Z 100016a0 f   vcom_proxy.obj
 0001:000008b0       ?AddJumpListTasks@SPVistaCOMProxy@@AAE_NPAUIObjectCollection@@PB_W@Z 100018b0 f   vcom_proxy.obj
 0001:00000a00       ?AddJumpListTask@SPVistaCOMProxy@@AAE_NPAUIObjectCollection@@PB_W1@Z 10001a00 f   vcom_proxy.obj
 0001:00000c80       ?AddJumpListSeparator@SPVistaCOMProxy@@AAE_NPAUIObjectCollection@@@Z 10001c80 f   vcom_proxy.obj
 0001:00000e20       _SetProgressState          10001e20 f   vcom_proxy.obj
 0001:00000e90       _SetProgressValue          10001e90 f   vcom_proxy.obj
 0001:00000f02       @__security_check_cookie@4 10001f02 f   LIBCMT:secchk.obj
 0001:00000f11       ??3@YAXPAX@Z               10001f11 f   LIBCMT:delete.obj
 0001:00000f1c       _wcsncpy                   10001f1c f   LIBCMT:wcsncpy.obj
 0001:00000f66       _wcstok                    10001f66 f   LIBCMT:wcstok.obj
 0001:00001011       ??1type_info@@UAE@XZ       10002011 f   LIBCMT:typinfo.obj
 0001:00001021       ??_Etype_info@@UAEPAXI@Z   10002021 f i LIBCMT:typinfo.obj
 0001:00001021       ??_Gtype_info@@UAEPAXI@Z   10002021 f i LIBCMT:typinfo.obj
 0001:00001042       ??8type_info@@QBE_NABV0@@Z 10002042 f   LIBCMT:typinfo.obj
 0001:0000111c       ___onexitinit              1000211c f   LIBCMT:onexit.obj
 0001:0000114d       __onexit                   1000214d f   LIBCMT:onexit.obj
 0001:00001189       _atexit                    10002189 f   LIBCMT:onexit.obj
 0001:000011a0       _wcsrchr                   100021a0 f   LIBCMT:wcsrchr.obj
 0001:000011cc       __CRT_INIT@12              100021cc f   LIBCMT:dllcrt0.obj
 0001:000013f7       __DllMainCRTStartup@12     100023f7 f   LIBCMT:dllcrt0.obj
 0001:0000141a       ___report_gsfailure        1000241a f   LIBCMT:gs_report.obj
 0001:00001520       _free                      10002520 f   LIBCMT:free.obj
 0001:000015ae       __encode_pointer           100025ae f   LIBCMT:tidtable.obj
 0001:00001620       __encoded_null             10002620 f   LIBCMT:tidtable.obj
 0001:00001629       __decode_pointer           10002629 f   LIBCMT:tidtable.obj
 0001:0000169b       ___crtTlsAlloc@4           1000269b f   LIBCMT:tidtable.obj
 0001:000016a4       ___set_flsgetvalue         100026a4 f   LIBCMT:tidtable.obj
 0001:000016d8       __mtterm                   100026d8 f   LIBCMT:tidtable.obj
 0001:00001715       __initptd                  10002715 f   LIBCMT:tidtable.obj
 0001:000017fc       __getptd_noexit            100027fc f   LIBCMT:tidtable.obj
 0001:00001875       __getptd                   10002875 f   LIBCMT:tidtable.obj
 0001:0000188f       __freefls@4                1000288f f   LIBCMT:tidtable.obj
 0001:000019be       __freeptd                  100029be f   LIBCMT:tidtable.obj
 0001:00001a2c       __mtinit                   10002a2c f   LIBCMT:tidtable.obj
 0001:00001bb9       ?_Type_info_dtor@type_info@@CAXPAV1@@Z 10002bb9 f   LIBCMT:typname.obj
 0001:00001c30       _strcmp                    10002c30 f   LIBCMT:strcmp.obj
 0001:00001cb8       __malloc_crt               10002cb8 f   LIBCMT:crtheap.obj
 0001:00001cfd       __calloc_crt               10002cfd f   LIBCMT:crtheap.obj
 0001:00001d49       __realloc_crt              10002d49 f   LIBCMT:crtheap.obj
 0001:00001d97       __msize                    10002d97 f   LIBCMT:msize.obj
 0001:00001e3a       __crt_waiting_on_module_handle 10002e3a f   LIBCMT:crt0dat.obj
 0001:00001e6a       __amsg_exit                10002e6a f   LIBCMT:crt0dat.obj
 0001:00001e93       ___crtCorExitProcess       10002e93 f   LIBCMT:crt0dat.obj
 0001:00001ebe       ___crtExitProcess          10002ebe f   LIBCMT:crt0dat.obj
 0001:00001ed6       __lockexit                 10002ed6 f   LIBCMT:crt0dat.obj
 0001:00001edf       __unlockexit               10002edf f   LIBCMT:crt0dat.obj
 0001:00001f05       __initterm_e               10002f05 f   LIBCMT:crt0dat.obj
 0001:00001f29       __cinit                    10002f29 f   LIBCMT:crt0dat.obj
 0001:000020da       __exit                     100030da f   LIBCMT:crt0dat.obj
 0001:000020f0       __cexit                    100030f0 f   LIBCMT:crt0dat.obj
 0001:000020ff       __init_pointers            100030ff f   LIBCMT:crt0dat.obj
 0001:00002150       __SEH_prolog4              10003150 f   LIBCMT:sehprolg4.obj
 0001:00002195       __SEH_epilog4              10003195 f   LIBCMT:sehprolg4.obj
 0001:000021b0       __except_handler4          100031b0 f   LIBCMT:chandler4.obj
 0001:0000233c       __ioinit                   1000333c f   LIBCMT:ioinit.obj
 0001:00002590       __ioterm                   10003590 f   LIBCMT:ioinit.obj
 0001:000025de       __setenvp                  100035de f   LIBCMT:stdenvp.obj
 0001:00002856       __setargv                  10003856 f   LIBCMT:stdargv.obj
 0001:00002911       ___crtGetEnvironmentStringsA 10003911 f   LIBCMT:a_env.obj
 0001:00002a48       __RTC_Initialize           10003a48 f   LIBCMT:_initsect_.obj
 0001:00002a6e       __RTC_Terminate            10003a6e f   LIBCMT:_initsect_.obj
 0001:00002a94       __heap_init                10003a94 f   LIBCMT:heapinit.obj
 0001:00002ac4       __heap_term                10003ac4 f   LIBCMT:heapinit.obj
 0001:00002b38       __initp_misc_winxfltr      10003b38 f   LIBCMT:winxfltr.obj
 0001:00002b39       __XcptFilter               10003b39 f   LIBCMT:winxfltr.obj
 0001:00002c99       ___CppXcptFilter           10003c99 f   LIBCMT:winxfltr.obj
 0001:00002cb9       ___security_init_cookie    10003cb9 f   LIBCMT:gs_support.obj
 0001:00002d4f       __crt_debugger_hook        10003d4f f   LIBCMT:dbghook.obj
 0001:00002d57       __get_errno_from_oserr     10003d57 f   LIBCMT:dosmap.obj
 0001:00002d99       __errno                    10003d99 f   LIBCMT:dosmap.obj
 0001:00002dac       __mtinitlocks              10003dac f   LIBCMT:mlock.obj
 0001:00002df7       __mtdeletelocks            10003df7 f   LIBCMT:mlock.obj
 0001:00002e4e       __unlock                   10003e4e f   LIBCMT:mlock.obj
 0001:00002e65       __mtinitlocknum            10003e65 f   LIBCMT:mlock.obj
 0001:00002f28       __lock                     10003f28 f   LIBCMT:mlock.obj
 0001:00002f5b       ___sbh_find_block          10003f5b f   LIBCMT:sbheap.obj
 0001:00002f8b       ___sbh_free_block          10003f8b f   LIBCMT:sbheap.obj
 0001:000032a1       ___sbh_alloc_new_region    100042a1 f   LIBCMT:sbheap.obj
 0001:00003351       ___sbh_alloc_new_group     10004351 f   LIBCMT:sbheap.obj
 0001:00003459       ___sbh_resize_block        10004459 f   LIBCMT:sbheap.obj
 0001:0000373a       ___sbh_alloc_block         1000473a f   LIBCMT:sbheap.obj
 0001:00003a1f       ___freetlocinfo            10004a1f f   LIBCMT:setlocal.obj
 0001:00003b68       ___addlocaleref            10004b68 f   LIBCMT:setlocal.obj
 0001:00003bf7       ___removelocaleref         10004bf7 f   LIBCMT:setlocal.obj
 0001:00003cce       ___updatetlocinfo          10004cce f   LIBCMT:setlocal.obj
 0001:00003f6a       ___updatetmbcinfo          10004f6a f   LIBCMT:mbctype.obj
 0001:0000400e       ??0_LocaleUpdate@@QAE@PAUlocaleinfo_struct@@@Z 1000500e f i LIBCMT:mbctype.obj
 0001:00004111       __setmbcp_nolock           10005111 f   LIBCMT:mbctype.obj
 0001:000042f6       __setmbcp                  100052f6 f   LIBCMT:mbctype.obj
 0001:00004490       ___initmbctable            10005490 f   LIBCMT:mbctype.obj
 0001:000044ae       __initp_misc_invarg        100054ae f   LIBCMT:invarg.obj
 0001:000044bd       __invoke_watson            100054bd f   LIBCMT:invarg.obj
 0001:000045e5       __invalid_parameter        100055e5 f   LIBCMT:invarg.obj
 0001:0000460b       _strcpy_s                  1000560b f   LIBCMT:strcpy_s.obj
 0001:00004680       _strlen                    10005680 f   LIBCMT:strlen.obj
 0001:0000470b       _V6_HeapAlloc              1000570b f   LIBCMT:malloc.obj
 0001:0000475a       _malloc                    1000575a f   LIBCMT:malloc.obj
 0001:00004824       __local_unwind4            10005824 f   LIBCMT:exsup4.obj
 0001:000048fa       __seh_longjmp_unwind4@4    100058fa f   LIBCMT:exsup4.obj
 0001:00004916       @_EH4_CallFilterFunc@8     10005916 f   LIBCMT:exsup4.obj
 0001:0000492d       @_EH4_TransferToHandler@8  1000592d f   LIBCMT:exsup4.obj
 0001:00004946       @_EH4_GlobalUnwind@4       10005946 f   LIBCMT:exsup4.obj
 0001:00004960       @_EH4_LocalUnwind@16       10005960 f   LIBCMT:exsup4.obj
 0001:00004977       __calloc_impl              10005977 f   LIBCMT:calloc_impl.obj
 0001:00004a95       _realloc                   10005a95 f   LIBCMT:realloc.obj
 0001:00004cb0       __NMSG_WRITE               10005cb0 f   LIBCMT:crt0msg.obj
 0001:00004e5b       __FF_MSGBANNER             10005e5b f   LIBCMT:crt0msg.obj
 0001:00004e94       __initp_misc_cfltcvt_tab   10005e94 f   LIBCMT:cmiscdat.obj
 0001:00004ec0       __ValidateImageBase        10005ec0 f   LIBCMT:pesect.obj
 0001:00004f00       __FindPESection            10005f00 f   LIBCMT:pesect.obj
 0001:00004f50       __IsNonwritableInCurrentImage 10005f50 f   LIBCMT:pesect.obj
 0001:0000500d       ?terminate@@YAXXZ          1000600d f   LIBCMT:hooks.obj
 0001:00005046       ?unexpected@@YAXXZ         10006046 f   LIBCMT:hooks.obj
 0001:00005059       ?_inconsistency@@YAXXZ     10006059 f   LIBCMT:hooks.obj
 0001:00005091       __initp_eh_hooks           10006091 f   LIBCMT:hooks.obj
 0001:000050a2       __initp_misc_winsig        100060a2 f   LIBCMT:winsig.obj
 0001:000050f7       ___get_sigabrt             100060f7 f   LIBCMT:winsig.obj
 0001:00005104       _raise                     10006104 f   LIBCMT:winsig.obj
 0001:000052b4       __initp_misc_rand_s        100062b4 f   LIBCMT:rand_s.obj
 0001:000052c3       __initp_misc_purevirt      100062c3 f   LIBCMT:inithelp.obj
 0001:000052d2       __initp_misc_initcrit      100062d2 f   LIBCMT:initcrit.obj
 0001:000052e1       ___crtInitCritSecAndSpinCount 100062e1 f   LIBCMT:initcrit.obj
 0001:00005341       __initp_heap_handler       10006341 f   LIBCMT:handler.obj
 0001:00005350       __callnewh                 10006350 f   LIBCMT:handler.obj
 0001:000053cb       __ismbblead                100063cb f   LIBCMT:ismbbyte.obj
 0001:000053f0       _memcpy                    100063f0 f   LIBCMT:memcpy.obj
 0001:00005760       _memmove                   10006760 f   LIBCMT:memmove.obj
 0001:00005ac5       ___free_lc_time            10006ac5 f   LIBCMT:inittime.obj
 0001:00005c5a       ___free_lconv_num          10006c5a f   LIBCMT:initnum.obj
 0001:00005c9f       ___free_lconv_mon          10006c9f f   LIBCMT:initmon.obj
 0001:00005d2d       __freea                    10006d2d f i LIBCMT:strftime.obj
 0001:00005d4d       _strcat_s                  10006d4d f   LIBCMT:strcat_s.obj
 0001:00005dd0       _strcspn                   10006dd0 f   LIBCMT:strcspn.obj
 0001:00005e16       _strncpy_s                 10006e16 f   LIBCMT:strncpy_s.obj
 0001:00005ed0       _memset                    10006ed0 f   LIBCMT:memset.obj
 0001:00006104       ___crtGetStringTypeA       10007104 f   LIBCMT:a_str.obj
 0001:00006150       _strpbrk                   10007150 f   LIBCMT:strpbrk.obj
 0001:00006535       ___crtLCMapStringA         10007535 f   LIBCMT:a_map.obj
 0001:00006580       __aulldvrm                 10007580 f   LIBCMT:ulldvrm.obj
 0001:00006620       __allmul                   10007620 f   LIBCMT:llmul.obj
 0001:00006654       _atol                      10007654 f   LIBCMT:atox.obj
 0001:0000666c       __global_unwind2           1000766c f   LIBCMT:exsup.obj
 0001:000066d1       __local_unwind2            100076d1 f   LIBCMT:exsup.obj
 0001:00006755       __abnormal_termination     10007755 f   LIBCMT:exsup.obj
 0001:00006778       __NLG_Notify1              10007778 f   LIBCMT:exsup.obj
 0001:00006781       __NLG_Notify               10007781 f   LIBCMT:exsup.obj
 0001:00006798       __NLG_Dispatch             10007798     LIBCMT:exsup.obj
 0001:00006798       __NLG_Dispatch2            10007798     LIBCMT:exsup.obj
 0001:000067a0       __NLG_Call                 100077a0 f   LIBCMT:exsup.obj
 0001:000067a2       __NLG_Return2              100077a2     LIBCMT:exsup.obj
 0001:000067a3       ___crtMessageBoxA          100077a3 f   LIBCMT:crtmbox.obj
 0001:0000690c       __set_error_mode           1000790c f   LIBCMT:errmode.obj
 0001:00006957       __fptrap                   10007957 f   LIBCMT:crt0fp.obj
 0001:00006960       _abort                     10007960 f   LIBCMT:abort.obj
 0001:00006afe       __VEC_memcpy               10007afe f   LIBCMT:p4_memcpy.obj
 0001:00006c31       __get_sse2_info            10007c31 f   LIBCMT:cpu_disp.obj
 0001:00006c93       ___sse2_available_init     10007c93 f   LIBCMT:cpu_disp.obj
 0001:00006ca0       __isleadbyte_l             10007ca0 f i LIBCMT:_wctype.obj
 0001:00006ce0       __alloca_probe_16          10007ce0 f   LIBCMT:alloca16.obj
 0001:00006cf6       __alloca_probe_8           10007cf6     LIBCMT:alloca16.obj
 0001:00006d63       __VEC_memzero              10007d63 f   LIBCMT:p4_memset.obj
 0001:00006df2       ___ansicp                  10007df2 f   LIBCMT:convrtcp.obj
 0001:00006e3b       ___convertcp               10007e3b f   LIBCMT:convrtcp.obj
 0001:0000721e       _strtol                    1000821e f   LIBCMT:strtol.obj
 0001:00007249       __isctype_l                10008249 f   LIBCMT:isctype.obj
 0001:00007310       __chkstk                   10008310 f   LIBCMT:chkstk.obj
 0001:00007310       __alloca_probe             10008310     LIBCMT:chkstk.obj
 0001:00007340       ___ascii_strnicmp          10008340 f   LIBCMT:_strnicm.obj
 0001:000073c0       _strchr                    100083c0 f   LIBCMT:strchr.obj
 0001:000073c6       ___from_strstr_to_strchr   100083c6     LIBCMT:strchr.obj
 0001:0000747e       _RtlUnwind@16              1000847e f   kernel32:KERNEL32.dll
 0001:00007484       ?_JumpToContinuation@@YGXPAXPAUEHRegistrationNode@@@Z 10008484 f   LIBCMT:_trnsctrl_.obj
 0001:000074b6       ?_CallMemberFunction0@@YGXPAX0@Z 100084b6 f   LIBCMT:_trnsctrl_.obj
 0001:000074b6       ?_CallMemberFunction1@@YGXPAX00@Z 100084b6 f   LIBCMT:_trnsctrl_.obj
 0001:000074b6       ?_CallMemberFunction2@@YGXPAX00H@Z 100084b6 f   LIBCMT:_trnsctrl_.obj
 0001:000074bd       ?_UnwindNestedFrames@@YGXPAUEHRegistrationNode@@PAUEHExceptionRecord@@@Z 100084bd f   LIBCMT:_trnsctrl_.obj
 0001:00007511       ___CxxFrameHandler3        10008511 f   LIBCMT:_trnsctrl_.obj
 0001:0000757a       ?_CallSETranslator@@YAHPAUEHExceptionRecord@@PAUEHRegistrationNode@@PAX2PBU_s_FuncInfo@@H1@Z 1000857a f   LIBCMT:_trnsctrl_.obj
 0001:000076f0       ?_GetRangeOfTrysToCheck@@YAPBU_s_TryBlockMapEntry@@PBU_s_FuncInfo@@HHPAI1@Z 100086f0 f   LIBCMT:_trnsctrl_.obj
 0001:00007765       __CreateFrameInfo          10008765 f   LIBCMT:_trnsctrl_.obj
 0001:00007791       __IsExceptionObjectToBeDestroyed 10008791 f   LIBCMT:_trnsctrl_.obj
 0001:000077b8       __FindAndUnlinkFrame       100087b8 f   LIBCMT:_trnsctrl_.obj
 0001:0000780a       ?_CallCatchBlock2@@YAPAXPAUEHRegistrationNode@@PBU_s_FuncInfo@@PAXHK@Z 1000880a f   LIBCMT:_trnsctrl_.obj
 0001:0000786a       ??0bad_exception@std@@QAE@PBD@Z 1000886a f i LIBCMT:frame.obj
 0001:00007888       ??1bad_exception@std@@UAE@XZ 10008888 f i LIBCMT:frame.obj
 0001:00007893       ??_Ebad_exception@std@@UAEPAXI@Z 10008893 f i LIBCMT:frame.obj
 0001:00007893       ??_Gbad_exception@std@@UAEPAXI@Z 10008893 f i LIBCMT:frame.obj
 0001:000078ba       ___TypeMatch               100088ba f   LIBCMT:frame.obj
 0001:00007919       ___FrameUnwindFilter       10008919 f   LIBCMT:frame.obj
 0001:00007962       ___FrameUnwindToState      10008962 f   LIBCMT:frame.obj
 0001:00007a88       ___DestructExceptionObject 10008a88 f   LIBCMT:frame.obj
 0001:00007add       ___AdjustPointer           10008add f   LIBCMT:frame.obj
 0001:00007d66       ___BuildCatchObjectHelper  10008d66 f   LIBCMT:frame.obj
 0001:00007ee5       ___BuildCatchObject        10008ee5 f   LIBCMT:frame.obj
 0001:00008420       ??0bad_exception@std@@QAE@ABV01@@Z 10009420 f i LIBCMT:frame.obj
 0001:0000843d       ___InternalCxxFrameHandler 1000943d f   LIBCMT:frame.obj
 0001:00008530       __CallSettingFrame@12      10009530 f   LIBCMT:lowhelpr.obj
 0001:00008557       __NLG_Return               10009557     LIBCMT:lowhelpr.obj
 0001:0000857c       ??0exception@std@@QAE@ABQBD@Z 1000957c f   LIBCMT:stdexcpt.obj
 0001:000085cf       ??0exception@std@@QAE@ABV01@@Z 100095cf f   LIBCMT:stdexcpt.obj
 0001:0000862c       ??1exception@std@@UAE@XZ   1000962c f   LIBCMT:stdexcpt.obj
 0001:00008642       ?what@exception@std@@UBEPBDXZ 10009642 f   LIBCMT:stdexcpt.obj
 0001:0000864f       ??_Gexception@std@@UAEPAXI@Z 1000964f f i LIBCMT:stdexcpt.obj
 0001:0000864f       ??_Eexception@std@@UAEPAXI@Z 1000964f f i LIBCMT:stdexcpt.obj
 0001:00008670       __EH_prolog3_catch         10009670 f   LIBCMT:ehprolg3.obj
 0001:000086a6       __CxxThrowException@8      100096a6 f   LIBCMT:throw.obj
 0001:000086f2       ?_ValidateRead@@YAHPBXI@Z  100096f2 f   LIBCMT:validate.obj
 0001:000086f2       ?_ValidateExecute@@YAHP6GHXZ@Z 100096f2 f   LIBCMT:validate.obj
 0001:000086f2       ?_ValidateWrite@@YAHPAXI@Z 100096f2 f   LIBCMT:validate.obj
 0002:00000000       __imp__GetModuleFileNameW@12 1000a000     kernel32:KERNEL32.dll
 0002:00000004       __imp__LCMapStringW@24     1000a004     kernel32:KERNEL32.dll
 0002:00000008       __imp__LCMapStringA@24     1000a008     kernel32:KERNEL32.dll
 0002:0000000c       __imp__GetStringTypeW@16   1000a00c     kernel32:KERNEL32.dll
 0002:00000010       __imp__GetCurrentThreadId@0 1000a010     kernel32:KERNEL32.dll
 0002:00000014       __imp__GetCommandLineA@0   1000a014     kernel32:KERNEL32.dll
 0002:00000018       __imp__TerminateProcess@8  1000a018     kernel32:KERNEL32.dll
 0002:0000001c       __imp__GetCurrentProcess@0 1000a01c     kernel32:KERNEL32.dll
 0002:00000020       __imp__UnhandledExceptionFilter@4 1000a020     kernel32:KERNEL32.dll
 0002:00000024       __imp__SetUnhandledExceptionFilter@4 1000a024     kernel32:KERNEL32.dll
 0002:00000028       __imp__IsDebuggerPresent@0 1000a028     kernel32:KERNEL32.dll
 0002:0000002c       __imp__GetLastError@0      1000a02c     kernel32:KERNEL32.dll
 0002:00000030       __imp__HeapFree@12         1000a030     kernel32:KERNEL32.dll
 0002:00000034       __imp__GetModuleHandleW@4  1000a034     kernel32:KERNEL32.dll
 0002:00000038       __imp__GetProcAddress@8    1000a038     kernel32:KERNEL32.dll
 0002:0000003c       __imp__TlsGetValue@4       1000a03c     kernel32:KERNEL32.dll
 0002:00000040       __imp__TlsAlloc@0          1000a040     kernel32:KERNEL32.dll
 0002:00000044       __imp__TlsSetValue@8       1000a044     kernel32:KERNEL32.dll
 0002:00000048       __imp__TlsFree@4           1000a048     kernel32:KERNEL32.dll
 0002:0000004c       __imp__InterlockedIncrement@4 1000a04c     kernel32:KERNEL32.dll
 0002:00000050       __imp__SetLastError@4      1000a050     kernel32:KERNEL32.dll
 0002:00000054       __imp__InterlockedDecrement@4 1000a054     kernel32:KERNEL32.dll
 0002:00000058       __imp__Sleep@4             1000a058     kernel32:KERNEL32.dll
 0002:0000005c       __imp__HeapSize@12         1000a05c     kernel32:KERNEL32.dll
 0002:00000060       __imp__ExitProcess@4       1000a060     kernel32:KERNEL32.dll
 0002:00000064       __imp__SetHandleCount@4    1000a064     kernel32:KERNEL32.dll
 0002:00000068       __imp__GetStdHandle@4      1000a068     kernel32:KERNEL32.dll
 0002:0000006c       __imp__GetFileType@4       1000a06c     kernel32:KERNEL32.dll
 0002:00000070       __imp__GetStartupInfoA@4   1000a070     kernel32:KERNEL32.dll
 0002:00000074       __imp__DeleteCriticalSection@4 1000a074     kernel32:KERNEL32.dll
 0002:00000078       __imp__GetModuleFileNameA@12 1000a078     kernel32:KERNEL32.dll
 0002:0000007c       __imp__FreeEnvironmentStringsA@4 1000a07c     kernel32:KERNEL32.dll
 0002:00000080       __imp__GetEnvironmentStrings@0 1000a080     kernel32:KERNEL32.dll
 0002:00000084       __imp__FreeEnvironmentStringsW@4 1000a084     kernel32:KERNEL32.dll
 0002:00000088       __imp__WideCharToMultiByte@32 1000a088     kernel32:KERNEL32.dll
 0002:0000008c       __imp__GetEnvironmentStringsW@0 1000a08c     kernel32:KERNEL32.dll
 0002:00000090       __imp__HeapCreate@12       1000a090     kernel32:KERNEL32.dll
 0002:00000094       __imp__HeapDestroy@4       1000a094     kernel32:KERNEL32.dll
 0002:00000098       __imp__VirtualFree@12      1000a098     kernel32:KERNEL32.dll
 0002:0000009c       __imp__QueryPerformanceCounter@4 1000a09c     kernel32:KERNEL32.dll
 0002:000000a0       __imp__GetTickCount@0      1000a0a0     kernel32:KERNEL32.dll
 0002:000000a4       __imp__GetCurrentProcessId@0 1000a0a4     kernel32:KERNEL32.dll
 0002:000000a8       __imp__GetSystemTimeAsFileTime@4 1000a0a8     kernel32:KERNEL32.dll
 0002:000000ac       __imp__LeaveCriticalSection@4 1000a0ac     kernel32:KERNEL32.dll
 0002:000000b0       __imp__EnterCriticalSection@4 1000a0b0     kernel32:KERNEL32.dll
 0002:000000b4       __imp__HeapAlloc@12        1000a0b4     kernel32:KERNEL32.dll
 0002:000000b8       __imp__VirtualAlloc@16     1000a0b8     kernel32:KERNEL32.dll
 0002:000000bc       __imp__HeapReAlloc@16      1000a0bc     kernel32:KERNEL32.dll
 0002:000000c0       __imp__GetCPInfo@8         1000a0c0     kernel32:KERNEL32.dll
 0002:000000c4       __imp__GetACP@0            1000a0c4     kernel32:KERNEL32.dll
 0002:000000c8       __imp__GetOEMCP@0          1000a0c8     kernel32:KERNEL32.dll
 0002:000000cc       __imp__IsValidCodePage@4   1000a0cc     kernel32:KERNEL32.dll
 0002:000000d0       __imp__RtlUnwind@16        1000a0d0     kernel32:KERNEL32.dll
 0002:000000d4       __imp__WriteFile@20        1000a0d4     kernel32:KERNEL32.dll
 0002:000000d8       __imp__LoadLibraryA@4      1000a0d8     kernel32:KERNEL32.dll
 0002:000000dc       __imp__InitializeCriticalSectionAndSpinCount@8 1000a0dc     kernel32:KERNEL32.dll
 0002:000000e0       __imp__GetLocaleInfoA@16   1000a0e0     kernel32:KERNEL32.dll
 0002:000000e4       __imp__GetStringTypeA@20   1000a0e4     kernel32:KERNEL32.dll
 0002:000000e8       __imp__MultiByteToWideChar@24 1000a0e8     kernel32:KERNEL32.dll
 0002:000000ec       __imp__RaiseException@16   1000a0ec     kernel32:KERNEL32.dll
 0002:000000f0       \177KERNEL32_NULL_THUNK_DATA 1000a0f0     kernel32:KERNEL32.dll
 0002:000000f4       __imp__SHCreateItemFromParsingName@16 1000a0f4     shell32:SHELL32.dll
 0002:000000f8       \177SHELL32_NULL_THUNK_DATA 1000a0f8     shell32:SHELL32.dll
 0002:000000fc       __imp__SHStrDupW@8         1000a0fc     shlwapi:SHLWAPI.dll
 0002:00000100       \177SHLWAPI_NULL_THUNK_DATA 1000a100     shlwapi:SHLWAPI.dll
 0002:00000104       __imp__PropVariantClear@4  1000a104     ole32:ole32.dll
 0002:00000108       __imp__CoCreateInstance@20 1000a108     ole32:ole32.dll
 0002:0000010c       __imp__CoTaskMemFree@4     1000a10c     ole32:ole32.dll
 0002:00000110       \177ole32_NULL_THUNK_DATA  1000a110     ole32:ole32.dll
 0002:00000114       ___xc_a                    1000a114     LIBCMT:crt0init.obj
 0002:00000118       ___xc_z                    1000a118     LIBCMT:crt0init.obj
 0002:0000011c       ___xi_a                    1000a11c     LIBCMT:crt0init.obj
 0002:0000012c       ___xi_z                    1000a12c     LIBCMT:crt0init.obj
 0002:00000130       ___xp_a                    1000a130     LIBCMT:crt0init.obj
 0002:00000134       ___xp_z                    1000a134     LIBCMT:crt0init.obj
 0002:00000138       ___xt_a                    1000a138     LIBCMT:crt0init.obj
 0002:0000013c       ___xt_z                    1000a13c     LIBCMT:crt0init.obj
 0002:00000140       _CLSID_ShellLink           1000a140     uuid:shguids2.obj
 0002:00000150       _CLSID_TaskbarList         1000a150     uuid:shguids2.obj
 0002:00000160       _CLSID_DestinationList     1000a160     uuid:shguids2.obj
 0002:00000170       _CLSID_EnumerableObjectCollection 1000a170     uuid:shguids2.obj
 0002:00000180       _PKEY_Title                1000a180     uuid:guids.obj
 0002:00000194       _PKEY_AppUserModel_IsDestListSeparator 1000a194     uuid:guids.obj
 0002:000001a8       ??_C@_0P@GHFPNOJB@bad?5allocation?$AA@ 1000a1a8     LIBCMT:typinfo.obj
 0002:000001bc       ??_7type_info@@6B@         1000a1bc     LIBCMT:typinfo.obj
 0002:000001c0       __pDefaultRawDllMain       1000a1c0     LIBCMT:dllcrt0.obj
 0002:000001c0       __pRawDllMain              1000a1c0     LIBCMT:dllcrt0.obj
 0002:000001cc       ??_C@_0O@NLDKAIKN@EncodePointer?$AA@ 1000a1cc     LIBCMT:tidtable.obj
 0002:000001dc       ??_C@_1BK@DBDEIDLH@?$AAK?$AAE?$AAR?$AAN?$AAE?$AAL?$AA3?$AA2?$AA?4?$AAD?$AAL?$AAL?$AA?$AA@ 1000a1dc     LIBCMT:tidtable.obj
 0002:000001f8       ??_C@_0O@KBPMFGHI@DecodePointer?$AA@ 1000a1f8     LIBCMT:tidtable.obj
 0002:00000208       ??_C@_07PEJMOBNF@FlsFree?$AA@ 1000a208     LIBCMT:tidtable.obj
 0002:00000210       ??_C@_0M@JCPCPOEF@FlsSetValue?$AA@ 1000a210     LIBCMT:tidtable.obj
 0002:0000021c       ??_C@_0M@GDNOONDI@FlsGetValue?$AA@ 1000a21c     LIBCMT:tidtable.obj
 0002:00000228       ??_C@_08KNHFBNJ@FlsAlloc?$AA@ 1000a228     LIBCMT:tidtable.obj
 0002:00000234       ??_C@_0P@MIGLKIOC@CorExitProcess?$AA@ 1000a234     LIBCMT:crt0dat.obj
 0002:00000244       ??_C@_1BI@BGOHAHKC@?$AAm?$AAs?$AAc?$AAo?$AAr?$AAe?$AAe?$AA?4?$AAd?$AAl?$AAl?$AA?$AA@ 1000a244     LIBCMT:crt0dat.obj
 0002:00000260       __XcptActTab               1000a260     LIBCMT:winxfltr.obj
 0002:00000358       ??_C@_01NEMOKFLO@?$DN?$AA@ 1000a358     LIBCMT:setlocal.obj
 0002:0000035a       ??_C@_00CNPNBAHC@?$AA@     1000a35a     LIBCMT:setlocal.obj
 0002:0000035c       ??_C@_0BK@CFCOFLF@?5Complete?5Object?5Locator?8?$AA@ 1000a35c     LIBCMT:undname.obj
 0002:00000378       ??_C@_0BN@MECKDCOJ@?5Class?5Hierarchy?5Descriptor?8?$AA@ 1000a378     LIBCMT:undname.obj
 0002:00000398       ??_C@_0BD@LGICGFMM@?5Base?5Class?5Array?8?$AA@ 1000a398     LIBCMT:undname.obj
 0002:000003ac       ??_C@_0BM@LDKODKLH@?5Base?5Class?5Descriptor?5at?5?$CI?$AA@ 1000a3ac     LIBCMT:undname.obj
 0002:000003c8       ??_C@_0BC@DAFEJGAK@?5Type?5Descriptor?8?$AA@ 1000a3c8     LIBCMT:undname.obj
 0002:000003dc       ??_C@_0BM@PMGGMLDN@?$GAlocal?5static?5thread?5guard?8?$AA@ 1000a3dc     LIBCMT:undname.obj
 0002:000003f8       ??_C@_0CL@FGIJHLCE@?$GAmanaged?5vector?5copy?5constructor@ 1000a3f8     LIBCMT:undname.obj
 0002:00000424       ??_C@_0CJ@GJELGAMM@?$GAvector?5vbase?5copy?5constructor?5i@ 1000a424     LIBCMT:undname.obj
 0002:00000450       ??_C@_0CD@CGAJBKEJ@?$GAvector?5copy?5constructor?5iterato@ 1000a450     LIBCMT:undname.obj
 0002:00000474       ??_C@_0CB@PDBIFEP@?$GAdynamic?5atexit?5destructor?5for?5?8@ 1000a474     LIBCMT:undname.obj
 0002:00000498       ??_C@_0BL@CLIPGLGB@?$GAdynamic?5initializer?5for?5?8?$AA@ 1000a498     LIBCMT:undname.obj
 0002:000004b4       ??_C@_0CM@FCBBDIGB@?$GAeh?5vector?5vbase?5copy?5constructo@ 1000a4b4     LIBCMT:undname.obj
 0002:000004e0       ??_C@_0CG@HLDDJMAG@?$GAeh?5vector?5copy?5constructor?5iter@ 1000a4e0     LIBCMT:undname.obj
 0002:00000508       ??_C@_0CF@IMGKMJNO@?$GAmanaged?5vector?5destructor?5itera@ 1000a508     LIBCMT:undname.obj
 0002:00000530       ??_C@_0CG@CFDHKGGD@?$GAmanaged?5vector?5constructor?5iter@ 1000a530     LIBCMT:undname.obj
 0002:00000558       ??_C@_0BN@CKNJLHMB@?$GAplacement?5delete?$FL?$FN?5closure?8?$AA@ 1000a558     LIBCMT:undname.obj
 0002:00000578       ??_C@_0BL@CNOONJFP@?$GAplacement?5delete?5closure?8?$AA@ 1000a578     LIBCMT:undname.obj
 0002:00000594       ??_C@_0P@HJKNJFNN@?$GAomni?5callsig?8?$AA@ 1000a594     LIBCMT:undname.obj
 0002:000005a4       ??_C@_09LBNFPBCA@?5delete?$FL?$FN?$AA@ 1000a5a4     LIBCMT:undname.obj
 0002:000005b0       ??_C@_06FHBGPFGH@?5new?$FL?$FN?$AA@ 1000a5b0     LIBCMT:undname.obj
 0002:000005b8       ??_C@_0CE@IIHCMGGL@?$GAlocal?5vftable?5constructor?5closu@ 1000a5b8     LIBCMT:undname.obj
 0002:000005dc       ??_C@_0BA@KKLDJDLB@?$GAlocal?5vftable?8?$AA@ 1000a5dc     LIBCMT:undname.obj
 0002:000005ec       ??_C@_05KHLCHHI@?$GARTTI?$AA@ 1000a5ec     LIBCMT:undname.obj
 0002:000005f4       ??_C@_03KLGMFNMG@?$GAEH?$AA@ 1000a5f4     LIBCMT:undname.obj
 0002:000005f8       ??_C@_0BA@KBCDOMBN@?$GAudt?5returning?8?$AA@ 1000a5f8     LIBCMT:undname.obj
 0002:00000608       ??_C@_0BL@LLKPOHJI@?$GAcopy?5constructor?5closure?8?$AA@ 1000a608     LIBCMT:undname.obj
 0002:00000624       ??_C@_0CH@OOJPLCPH@?$GAeh?5vector?5vbase?5constructor?5ite@ 1000a624     LIBCMT:undname.obj
 0002:0000064c       ??_C@_0CA@GCEOPDGL@?$GAeh?5vector?5destructor?5iterator?8?$AA@ 1000a64c     LIBCMT:undname.obj
 0002:0000066c       ??_C@_0CB@JONCMFFK@?$GAeh?5vector?5constructor?5iterator?8@ 1000a66c     LIBCMT:undname.obj
 0002:00000690       ??_C@_0BL@NILFHHPC@?$GAvirtual?5displacement?5map?8?$AA@ 1000a690     LIBCMT:undname.obj
 0002:000006ac       ??_C@_0CE@IKBNEHA@?$GAvector?5vbase?5constructor?5iterat@ 1000a6ac     LIBCMT:undname.obj
 0002:000006d0       ??_C@_0BN@LFPFMEDL@?$GAvector?5destructor?5iterator?8?$AA@ 1000a6d0     LIBCMT:undname.obj
 0002:000006f0       ??_C@_0BO@PFGOCPJJ@?$GAvector?5constructor?5iterator?8?$AA@ 1000a6f0     LIBCMT:undname.obj
 0002:00000710       ??_C@_0BN@IMDCHIKM@?$GAscalar?5deleting?5destructor?8?$AA@ 1000a710     LIBCMT:undname.obj
 0002:00000730       ??_C@_0BO@OBMKPJIG@?$GAdefault?5constructor?5closure?8?$AA@ 1000a730     LIBCMT:undname.obj
 0002:00000750       ??_C@_0BN@DEGPLNFK@?$GAvector?5deleting?5destructor?8?$AA@ 1000a750     LIBCMT:undname.obj
 0002:00000770       ??_C@_0BD@JDLKDPAB@?$GAvbase?5destructor?8?$AA@ 1000a770     LIBCMT:undname.obj
 0002:00000784       ??_C@_08OBABFOLI@?$GAstring?8?$AA@ 1000a784     LIBCMT:undname.obj
 0002:00000790       ??_C@_0BF@KDPPACIK@?$GAlocal?5static?5guard?8?$AA@ 1000a790     LIBCMT:undname.obj
 0002:000007a8       ??_C@_08LLFFHHDJ@?$GAtypeof?8?$AA@ 1000a7a8     LIBCMT:undname.obj
 0002:000007b4       ??_C@_07FEEIOKP@?$GAvcall?8?$AA@ 1000a7b4     LIBCMT:undname.obj
 0002:000007bc       ??_C@_09BLBHBJP@?$GAvbtable?8?$AA@ 1000a7bc     LIBCMT:undname.obj
 0002:000007c8       ??_C@_09IFPLHPGF@?$GAvftable?8?$AA@ 1000a7c8     LIBCMT:undname.obj
 0002:000007d4       ??_C@_02MHEGNOJ@?$FO?$DN?$AA@ 1000a7d4     LIBCMT:undname.obj
 0002:000007d8       ??_C@_02DHLNPPGH@?$HM?$DN?$AA@ 1000a7d8     LIBCMT:undname.obj
 0002:000007dc       ??_C@_02FGJGFEAB@?$CG?$DN?$AA@ 1000a7dc     LIBCMT:undname.obj
 0002:000007e0       ??_C@_03CDNPDDLA@?$DM?$DM?$DN?$AA@ 1000a7e0     LIBCMT:undname.obj
 0002:000007e4       ??_C@_03IKFCCPFF@?$DO?$DO?$DN?$AA@ 1000a7e4     LIBCMT:undname.obj
 0002:000007e8       ??_C@_02FENAOKFI@?$CF?$DN?$AA@ 1000a7e8     LIBCMT:undname.obj
 0002:000007ec       ??_C@_02FJEHGPIO@?1?$DN?$AA@ 1000a7ec     LIBCMT:undname.obj
 0002:000007f0       ??_C@_02FKMDLLOA@?9?$DN?$AA@ 1000a7f0     LIBCMT:undname.obj
 0002:000007f4       ??_C@_02FOEOMHFC@?$CL?$DN?$AA@ 1000a7f4     LIBCMT:undname.obj
 0002:000007f8       ??_C@_02FPIMKNGF@?$CK?$DN?$AA@ 1000a7f8     LIBCMT:undname.obj
 0002:000007fc       ??_C@_02NONPIBCD@?$HM?$HM?$AA@ 1000a7fc     LIBCMT:undname.obj
 0002:00000800       ??_C@_02PPKAJPJL@?$CG?$CG?$AA@ 1000a800     LIBCMT:undname.obj
 0002:00000804       ??_C@_01DNKMNLPK@?$HM?$AA@ 1000a804     LIBCMT:undname.obj
 0002:00000808       ??_C@_01JKBOJNNK@?$FO?$AA@ 1000a808     LIBCMT:undname.obj
 0002:0000080c       ??_C@_01PJKLJHI@?$HO?$AA@  1000a80c     LIBCMT:undname.obj
 0002:00000810       ??_C@_02HCKGKOFO@?$CI?$CJ?$AA@ 1000a810     LIBCMT:undname.obj
 0002:00000814       ??_C@_01IHBHIGKO@?0?$AA@   1000a814     LIBCMT:undname.obj
 0002:00000818       ??_C@_02EEKDKGMJ@?$DO?$DN?$AA@ 1000a818     LIBCMT:undname.obj
 0002:0000081c       ??_C@_01PPODPGHN@?$DO?$AA@ 1000a81c     LIBCMT:undname.obj
 0002:00000820       ??_C@_02EHCHHCKH@?$DM?$DN?$AA@ 1000a820     LIBCMT:undname.obj
 0002:00000824       ??_C@_01MNNFJEPP@?$DM?$AA@ 1000a824     LIBCMT:undname.obj
 0002:00000828       ??_C@_01FGNFDNOH@?$CF?$AA@ 1000a828     LIBCMT:undname.obj
 0002:0000082c       ??_C@_01KMDKNFGN@?1?$AA@   1000a82c     LIBCMT:undname.obj
 0002:00000830       ??_C@_03MNHNFDLC@?9?$DO?$CK?$AA@ 1000a830     LIBCMT:undname.obj
 0002:00000834       ??_C@_01HNPIGOCE@?$CG?$AA@ 1000a834     LIBCMT:undname.obj
 0002:00000838       ??_C@_01MIFGBAGJ@?$CL?$AA@ 1000a838     LIBCMT:undname.obj
 0002:0000083c       ??_C@_01JOAMLHOP@?9?$AA@   1000a83c     LIBCMT:undname.obj
 0002:00000840       ??_C@_02BAABKJLB@?9?9?$AA@ 1000a840     LIBCMT:undname.obj
 0002:00000844       ??_C@_02ECNGHCIF@?$CL?$CL?$AA@ 1000a844     LIBCMT:undname.obj
 0002:00000848       ??_C@_01NBENCBCI@?$CK?$AA@ 1000a848     LIBCMT:undname.obj
 0002:0000084c       ??_C@_02HBOOOICD@?9?$DO?$AA@ 1000a84c     LIBCMT:undname.obj
 0002:00000850       ??_C@_08LHJFAFGD@operator?$AA@ 1000a850     LIBCMT:undname.obj
 0002:0000085c       ??_C@_02GPECMEKF@?$FL?$FN?$AA@ 1000a85c     LIBCMT:undname.obj
 0002:00000860       ??_C@_02FDNJECIE@?$CB?$DN?$AA@ 1000a860     LIBCMT:undname.obj
 0002:00000864       ??_C@_02EGOFBIJA@?$DN?$DN?$AA@ 1000a864     LIBCMT:undname.obj
 0002:00000868       ??_C@_01DCLJPIOD@?$CB?$AA@ 1000a868     LIBCMT:undname.obj
 0002:0000086c       ??_C@_02FODMEDOG@?$DM?$DM?$AA@ 1000a86c     LIBCMT:undname.obj
 0002:00000870       ??_C@_02GPIOPFAK@?$DO?$DO?$AA@ 1000a870     LIBCMT:undname.obj
 0002:00000874       ??_C@_07FPCDHGMM@?5delete?$AA@ 1000a874     LIBCMT:undname.obj
 0002:0000087c       ??_C@_04NIHEBCM@?5new?$AA@ 1000a87c     LIBCMT:undname.obj
 0002:00000884       ??_C@_0M@GFIIJFMG@__unaligned?$AA@ 1000a884     LIBCMT:undname.obj
 0002:00000890       ??_C@_0L@PILCLIHE@__restrict?$AA@ 1000a890     LIBCMT:undname.obj
 0002:0000089c       ??_C@_07JOMMBBKO@__ptr64?$AA@ 1000a89c     LIBCMT:undname.obj
 0002:000008a4       ??_C@_09HIJEGCPM@__clrcall?$AA@ 1000a8a4     LIBCMT:undname.obj
 0002:000008b0       ??_C@_0L@JMKHOMEK@__fastcall?$AA@ 1000a8b0     LIBCMT:undname.obj
 0002:000008bc       ??_C@_0L@NPHFGOKO@__thiscall?$AA@ 1000a8bc     LIBCMT:undname.obj
 0002:000008c8       ??_C@_09IFJBGAPI@__stdcall?$AA@ 1000a8c8     LIBCMT:undname.obj
 0002:000008d4       ??_C@_08GHMPAG@__pascal?$AA@ 1000a8d4     LIBCMT:undname.obj
 0002:000008e0       ??_C@_07KOLFKCDI@__cdecl?$AA@ 1000a8e0     LIBCMT:undname.obj
 0002:000008e8       ??_C@_08EHJDFFNH@__based?$CI?$AA@ 1000a8e8     LIBCMT:undname.obj
 0002:00000a78       ??_C@_03KHICJKCI@?4?4?4?$AA@ 1000aa78     LIBCMT:undname.obj
 0002:00000a7c       ??_C@_0P@GGKDKEEG@runtime?5error?5?$AA@ 1000aa7c     LIBCMT:crt0msg.obj
 0002:00000a8c       ??_C@_02PCIJFNDE@?$AN?6?$AA@ 1000aa8c     LIBCMT:crt0msg.obj
 0002:00000a90       ??_C@_0O@MJNIPGOH@TLOSS?5error?$AN?6?$AA@ 1000aa90     LIBCMT:crt0msg.obj
 0002:00000aa0       ??_C@_0N@BONNPDHF@SING?5error?$AN?6?$AA@ 1000aaa0     LIBCMT:crt0msg.obj
 0002:00000ab0       ??_C@_0P@MBDAJNE@DOMAIN?5error?$AN?6?$AA@ 1000aab0     LIBCMT:crt0msg.obj
 0002:00000ac0       ??_C@_0JL@DFDOOABL@R6034?$AN?6An?5application?5has?5made?5a@ 1000aac0     LIBCMT:crt0msg.obj
 0002:00000b60       ??_C@_0PH@EPAFIJ@R6033?$AN?6?9?5Attempt?5to?5use?5MSIL?5cod@ 1000ab60     LIBCMT:crt0msg.obj
 0002:00000c58       ??_C@_0DD@BKEEABMM@R6032?$AN?6?9?5not?5enough?5space?5for?5lo@ 1000ac58     LIBCMT:crt0msg.obj
 0002:00000c90       ??_C@_0GD@OFKILIED@R6031?$AN?6?9?5Attempt?5to?5initialize?5t@ 1000ac90     LIBCMT:crt0msg.obj
 0002:00000cf4       ??_C@_0BP@LPMHJOKI@R6030?$AN?6?9?5CRT?5not?5initialized?$AN?6?$AA@ 1000acf4     LIBCMT:crt0msg.obj
 0002:00000d14       ??_C@_0CF@KJDAIALP@R6028?$AN?6?9?5unable?5to?5initialize?5he@ 1000ad14     LIBCMT:crt0msg.obj
 0002:00000d3c       ??_C@_0DF@GAKBPDFP@R6027?$AN?6?9?5not?5enough?5space?5for?5lo@ 1000ad3c     LIBCMT:crt0msg.obj
 0002:00000d74       ??_C@_0DF@IBLNNAIG@R6026?$AN?6?9?5not?5enough?5space?5for?5st@ 1000ad74     LIBCMT:crt0msg.obj
 0002:00000dac       ??_C@_0CG@IOHKGFNJ@R6025?$AN?6?9?5pure?5virtual?5function?5c@ 1000adac     LIBCMT:crt0msg.obj
 0002:00000dd4       ??_C@_0DF@JIJJFJDC@R6024?$AN?6?9?5not?5enough?5space?5for?5_o@ 1000add4     LIBCMT:crt0msg.obj
 0002:00000e0c       ??_C@_0CJ@EGEJHFME@R6019?$AN?6?9?5unable?5to?5open?5console?5@ 1000ae0c     LIBCMT:crt0msg.obj
 0002:00000e38       ??_C@_0CB@GNHNIELH@R6018?$AN?6?9?5unexpected?5heap?5error?$AN?6@ 1000ae38     LIBCMT:crt0msg.obj
 0002:00000e5c       ??_C@_0CN@FOLDKNG@R6017?$AN?6?9?5unexpected?5multithread?5@ 1000ae5c     LIBCMT:crt0msg.obj
 0002:00000e8c       ??_C@_0CM@FAHFJNHO@R6016?$AN?6?9?5not?5enough?5space?5for?5th@ 1000ae8c     LIBCMT:crt0msg.obj
 0002:00000eb8       ??_C@_0JG@LBKMGKLD@?$AN?6This?5application?5has?5requested@ 1000aeb8     LIBCMT:crt0msg.obj
 0002:00000f50       ??_C@_0CM@FLCNIPKK@R6009?$AN?6?9?5not?5enough?5space?5for?5en@ 1000af50     LIBCMT:crt0msg.obj
 0002:00000f7c       ??_C@_0CK@KMMJOAPP@R6008?$AN?6?9?5not?5enough?5space?5for?5ar@ 1000af7c     LIBCMT:crt0msg.obj
 0002:00000fa8       ??_C@_0CN@LEKKICBM@R6002?$AN?6?9?5floating?5point?5support?5@ 1000afa8     LIBCMT:crt0msg.obj
 0002:00000fd8       ??_C@_0CF@GOGNBNAK@Microsoft?5Visual?5C?$CL?$CL?5Runtime?5Lib@ 1000afd8     LIBCMT:crt0msg.obj
 0002:00001000       ??_C@_02PHMGELLB@?6?6?$AA@ 1000b000     LIBCMT:crt0msg.obj
 0002:00001004       ??_C@_0BH@DNAGHKFM@?$DMprogram?5name?5unknown?$DO?$AA@ 1000b004     LIBCMT:crt0msg.obj
 0002:0000101c       ??_C@_0BK@OFGJDLJJ@Runtime?5Error?$CB?6?6Program?3?5?$AA@ 1000b01c     LIBCMT:crt0msg.obj
 0002:00001038       ___newctype                1000b038     LIBCMT:ctype.obj
 0002:00001338       __wctype                   1000b338     LIBCMT:ctype.obj
 0002:00001540       ___newclmap                1000b540     LIBCMT:ctype.obj
 0002:000016c0       ___newcumap                1000b6c0     LIBCMT:ctype.obj
 0002:00001840       ??_C@_08JCCMCCIL@HH?3mm?3ss?$AA@ 1000b840     LIBCMT:strftime.obj
 0002:0000184c       ??_C@_0BE@CKGJFCPC@dddd?0?5MMMM?5dd?0?5yyyy?$AA@ 1000b84c     LIBCMT:strftime.obj
 0002:00001860       ??_C@_08BPBNCDIB@MM?1dd?1yy?$AA@ 1000b860     LIBCMT:strftime.obj
 0002:0000186c       ??_C@_02CJNFDJBF@PM?$AA@   1000b86c     LIBCMT:strftime.obj
 0002:00001870       ??_C@_02DEDBPAFC@AM?$AA@   1000b870     LIBCMT:strftime.obj
 0002:00001874       ??_C@_08EDHMEBNP@December?$AA@ 1000b874     LIBCMT:strftime.obj
 0002:00001880       ??_C@_08HCHEGEOA@November?$AA@ 1000b880     LIBCMT:strftime.obj
 0002:0000188c       ??_C@_07JJNFCEND@October?$AA@ 1000b88c     LIBCMT:strftime.obj
 0002:00001894       ??_C@_09BHHEALKD@September?$AA@ 1000b894     LIBCMT:strftime.obj
 0002:000018a0       ??_C@_06LBBHFDDG@August?$AA@ 1000b8a0     LIBCMT:strftime.obj
 0002:000018a8       ??_C@_04MIEPOIFP@July?$AA@ 1000b8a8     LIBCMT:strftime.obj
 0002:000018b0       ??_C@_04CNLMGBGM@June?$AA@ 1000b8b0     LIBCMT:strftime.obj
 0002:000018b8       ??_C@_05DMJDNLEJ@April?$AA@ 1000b8b8     LIBCMT:strftime.obj
 0002:000018c0       ??_C@_05HPCKOFNC@March?$AA@ 1000b8c0     LIBCMT:strftime.obj
 0002:000018c8       ??_C@_08GNJGEPFN@February?$AA@ 1000b8c8     LIBCMT:strftime.obj
 0002:000018d4       ??_C@_07CGJPFGJA@January?$AA@ 1000b8d4     LIBCMT:strftime.obj
 0002:000018dc       ??_C@_03MKABNOCG@Dec?$AA@  1000b8dc     LIBCMT:strftime.obj
 0002:000018e0       ??_C@_03JPJOFNIA@Nov?$AA@  1000b8e0     LIBCMT:strftime.obj
 0002:000018e4       ??_C@_03BMAOKBAD@Oct?$AA@  1000b8e4     LIBCMT:strftime.obj
 0002:000018e8       ??_C@_03GGCAPAJC@Sep?$AA@  1000b8e8     LIBCMT:strftime.obj
 0002:000018ec       ??_C@_03IFJFEIGA@Aug?$AA@  1000b8ec     LIBCMT:strftime.obj
 0002:000018f0       ??_C@_03LBGABGKK@Jul?$AA@  1000b8f0     LIBCMT:strftime.obj
 0002:000018f4       ??_C@_03IDFGHECI@Jun?$AA@  1000b8f4     LIBCMT:strftime.obj
 0002:000018f8       ??_C@_03CNMDKL@May?$AA@    1000b8f8     LIBCMT:strftime.obj
 0002:000018fc       ??_C@_03LEOLGMJP@Apr?$AA@  1000b8fc     LIBCMT:strftime.obj
 0002:00001900       ??_C@_03ODNJBKGA@Mar?$AA@  1000b900     LIBCMT:strftime.obj
 0002:00001904       ??_C@_03HJBDCHOM@Feb?$AA@  1000b904     LIBCMT:strftime.obj
 0002:00001908       ??_C@_03JIHJHPIE@Jan?$AA@  1000b908     LIBCMT:strftime.obj
 0002:0000190c       ??_C@_08INBOOONO@Saturday?$AA@ 1000b90c     LIBCMT:strftime.obj
 0002:00001918       ??_C@_06JECMNKMI@Friday?$AA@ 1000b918     LIBCMT:strftime.obj
 0002:00001920       ??_C@_08HACCIKIA@Thursday?$AA@ 1000b920     LIBCMT:strftime.obj
 0002:0000192c       ??_C@_09DLIGFAKA@Wednesday?$AA@ 1000b92c     LIBCMT:strftime.obj
 0002:00001938       ??_C@_07BAAGCFCM@Tuesday?$AA@ 1000b938     LIBCMT:strftime.obj
 0002:00001940       ??_C@_06JLEDEDGH@Monday?$AA@ 1000b940     LIBCMT:strftime.obj
 0002:00001948       ??_C@_06OOPIFAJ@Sunday?$AA@ 1000b948     LIBCMT:strftime.obj
 0002:00001950       ??_C@_03FEFJNEK@Sat?$AA@   1000b950     LIBCMT:strftime.obj
 0002:00001954       ??_C@_03IDIOELNC@Fri?$AA@  1000b954     LIBCMT:strftime.obj
 0002:00001958       ??_C@_03IOFIKPDN@Thu?$AA@  1000b958     LIBCMT:strftime.obj
 0002:0000195c       ??_C@_03MHOMLAJA@Wed?$AA@  1000b95c     LIBCMT:strftime.obj
 0002:00001960       ??_C@_03NAGEINEP@Tue?$AA@  1000b960     LIBCMT:strftime.obj
 0002:00001964       ??_C@_03PDAGKDH@Mon?$AA@   1000b964     LIBCMT:strftime.obj
 0002:00001968       ??_C@_03KOEHGMDN@Sun?$AA@  1000b968     LIBCMT:strftime.obj
 0002:0000196c       ??_C@_13NOLLCAOD@?$AA?$AA?$AA?$AA@ 1000b96c     LIBCMT:a_str.obj
 0002:00001970       ??_C@_0BI@DFKBFLJE@GetProcessWindowStation?$AA@ 1000b970     LIBCMT:crtmbox.obj
 0002:00001988       ??_C@_0BK@CIDNPOGP@GetUserObjectInformationA?$AA@ 1000b988     LIBCMT:crtmbox.obj
 0002:000019a4       ??_C@_0BD@HHGDFDBJ@GetLastActivePopup?$AA@ 1000b9a4     LIBCMT:crtmbox.obj
 0002:000019b8       ??_C@_0BA@HNOPNCHB@GetActiveWindow?$AA@ 1000b9b8     LIBCMT:crtmbox.obj
 0002:000019c8       ??_C@_0M@CHKKJDAI@MessageBoxA?$AA@ 1000b9c8     LIBCMT:crtmbox.obj
 0002:000019d4       ??_C@_0L@NDEGIDAG@USER32?4DLL?$AA@ 1000b9d4     LIBCMT:crtmbox.obj
 0002:000019e0       ___dnames                  1000b9e0     LIBCMT:timeset.obj
 0002:000019f8       ___mnames                  1000b9f8     LIBCMT:timeset.obj
 0002:00001a30       ??_C@_13GGAHEHIG@?$AA?$AB?$AA?$AA@ 1000ba30     vcom_proxy.obj
 0002:00001a34       ??_C@_13IMODFHAA@?$AA?9?$AA?$AA@ 1000ba34     vcom_proxy.obj
 0002:00001a38       __GUID_43826d1e_e718_42ee_bc55_a1e261c37bfe 1000ba38     vcom_proxy.obj
 0002:00001a48       __GUID_c0b4e2f3_ba21_4773_8dba_335ec946eb8b 1000ba48     vcom_proxy.obj
 0002:00001a58       __GUID_dc1c5a9c_e88a_4dde_a5a1_60f82a20aef7 1000ba58     vcom_proxy.obj
 0002:00001a68       __GUID_92ca9dcd_5622_4bba_a805_5e9f541bd8c9 1000ba68     vcom_proxy.obj
 0002:00001a78       __GUID_886d8eeb_8cf2_4446_8d02_cdba1dbdcf99 1000ba78     vcom_proxy.obj
 0002:00001a88       __GUID_ea1afb91_9e28_4b86_90e9_9e9f8a5eefaf 1000ba88     vcom_proxy.obj
 0002:00001a98       __GUID_d57c7288_d4ad_4768_be02_9d969532d960 1000ba98     vcom_proxy.obj
 0002:00001aa8       __GUID_84bccd23_5fde_4cdb_aea4_af64b83d78ab 1000baa8     vcom_proxy.obj
 0002:00001ab8       __GUID_6332debf_87b5_4670_90c0_5e57b408a49e 1000bab8     vcom_proxy.obj
 0002:00001ac8       __GUID_5632b1a4_e38a_400a_928a_d4cd63230295 1000bac8     vcom_proxy.obj
 0002:00001ad8       __GUID_000214f9_0000_0000_c000_000000000046 1000bad8     vcom_proxy.obj
 0002:00001ae8       __pDestructExceptionObject 1000bae8     LIBCMT:frame.obj
 0002:00001af0       ??_7bad_exception@std@@6B@ 1000baf0     LIBCMT:frame.obj
 0002:00001af8       ??_C@_0O@DPKOEFFH@bad?5exception?$AA@ 1000baf8     LIBCMT:frame.obj
 0002:00001b0c       ??_7exception@std@@6B@     1000bb0c     LIBCMT:stdexcpt.obj
 0002:00001b14       ??_C@_0BC@EOODALEL@Unknown?5exception?$AA@ 1000bb14     LIBCMT:stdexcpt.obj
 0002:00001b48       __load_config_used         1000bb48     LIBCMT:loadcfg.obj
 0002:00001b90       ??_R4type_info@@6B@        1000bb90     LIBCMT:typinfo.obj
 0002:00001ba4       ??_R3type_info@@8          1000bba4     LIBCMT:typinfo.obj
 0002:00001bb4       ??_R2type_info@@8          1000bbb4     LIBCMT:typinfo.obj
 0002:00001bbc       ??_R1A@?0A@EA@type_info@@8 1000bbbc     LIBCMT:typinfo.obj
 0002:00001bd8       ??_R4bad_exception@std@@6B@ 1000bbd8     LIBCMT:frame.obj
 0002:00001bec       ??_R3bad_exception@std@@8  1000bbec     LIBCMT:frame.obj
 0002:00001bfc       ??_R2bad_exception@std@@8  1000bbfc     LIBCMT:frame.obj
 0002:00001c08       ??_R1A@?0A@EA@bad_exception@std@@8 1000bc08     LIBCMT:frame.obj
 0002:00001c24       ??_R1A@?0A@EA@exception@std@@8 1000bc24     LIBCMT:frame.obj
 0002:00001c40       ??_R3exception@std@@8      1000bc40     LIBCMT:frame.obj
 0002:00001c50       ??_R2exception@std@@8      1000bc50     LIBCMT:frame.obj
 0002:00001c58       ??_R4exception@std@@6B@    1000bc58     LIBCMT:stdexcpt.obj
 0002:00001c70       ___safe_se_handler_table   1000bc70     <linker-defined>
 0002:00001c98       ___rtc_iaa                 1000bc98     LIBCMT:_initsect_.obj
 0002:00001c9c       ___rtc_izz                 1000bc9c     LIBCMT:_initsect_.obj
 0002:00001ca0       ___rtc_taa                 1000bca0     LIBCMT:_initsect_.obj
 0002:00001ca4       ___rtc_tzz                 1000bca4     LIBCMT:_initsect_.obj
 0002:0000215c       __TI2?AVbad_exception@std@@ 1000c15c     LIBCMT:frame.obj
 0002:0000216c       __CTA2?AVbad_exception@std@@ 1000c16c     LIBCMT:frame.obj
 0002:00002178       __CT??_R0?AVbad_exception@std@@@8??0bad_exception@std@@QAE@ABV01@@Z12 1000c178     LIBCMT:frame.obj
 0002:00002194       __CT??_R0?AVexception@std@@@8??0exception@std@@QAE@ABV01@@Z12 1000c194     LIBCMT:frame.obj
 0002:000021b0       __IMPORT_DESCRIPTOR_KERNEL32 1000c1b0     kernel32:KERNEL32.dll
 0002:000021c4       __IMPORT_DESCRIPTOR_SHELL32 1000c1c4     shell32:SHELL32.dll
 0002:000021d8       __IMPORT_DESCRIPTOR_ole32  1000c1d8     ole32:ole32.dll
 0002:000021ec       __IMPORT_DESCRIPTOR_SHLWAPI 1000c1ec     shlwapi:SHLWAPI.dll
 0002:00002200       __NULL_IMPORT_DESCRIPTOR   1000c200     kernel32:KERNEL32.dll
 0003:00000004       ??_R0?AVtype_info@@@8      1000d004     LIBCMT:typinfo.obj
 0003:0000001c       ___security_cookie         1000d01c     LIBCMT:gs_cookie.obj
 0003:00000020       ___security_cookie_complement 1000d020     LIBCMT:gs_cookie.obj
 0003:00000024       ___flsindex                1000d024     LIBCMT:tidtable.obj
 0003:00000028       ___getvalueindex           1000d028     LIBCMT:tidtable.obj
 0003:00000030       __aexit_rtn                1000d030     LIBCMT:crt0dat.obj
 0003:00000038       ___badioinfo               1000d038     LIBCMT:ioinit.obj
 0003:00000078       __amblksiz                 1000d078     LIBCMT:heapinit.obj
 0003:0000007c       __First_FPE_Indx           1000d07c     LIBCMT:winxfltr.obj
 0003:00000080       __Num_FPE                  1000d080     LIBCMT:winxfltr.obj
 0003:00000084       __XcptActTabSize           1000d084     LIBCMT:winxfltr.obj
 0003:00000088       __XcptActTabCount          1000d088     LIBCMT:winxfltr.obj
 0003:00000328       ___clocalestr              1000d328     LIBCMT:nlsdata2.obj
 0003:00000330       ___initiallocinfo          1000d330     LIBCMT:nlsdata2.obj
 0003:00000408       ___ptlocinfo               1000d408     LIBCMT:nlsdata2.obj
 0003:0000040c       ___lc_clike                1000d40c     LIBCMT:nlsdata2.obj
 0003:00000410       ___initiallocalestructinfo 1000d410     LIBCMT:nlsdata2.obj
 0003:00000418       ___initialmbcinfo          1000d418     LIBCMT:mbctype.obj
 0003:00000638       __mbctype                  1000d638     LIBCMT:mbctype.obj
 0003:00000740       __mbcasemap                1000d740     LIBCMT:mbctype.obj
 0003:00000840       ___ptmbcinfo               1000d840     LIBCMT:mbctype.obj
 0003:000009f8       __cfltcvt_tab              1000d9f8     LIBCMT:cmiscdat.obj
 0003:00000a20       __pctype                   1000da20     LIBCMT:ctype.obj
 0003:00000a24       __pwctype                  1000da24     LIBCMT:ctype.obj
 0003:00000a28       ___lc_time_c               1000da28     LIBCMT:strftime.obj
 0003:00000ae0       ___lc_time_curr            1000dae0     LIBCMT:strftime.obj
 0003:00000ae4       ___lconv_static_decimal    1000dae4     LIBCMT:lconv.obj
 0003:00000ae8       ___lconv_c                 1000dae8     LIBCMT:lconv.obj
 0003:00000b18       ___lconv                   1000db18     LIBCMT:lconv.obj
 0003:00000b1c       ___globallocalestatus      1000db1c     LIBCMT:glstatus.obj
 0003:00000b20       ___mb_cur_max              1000db20     LIBCMT:nlsdata1.obj
 0003:00000b24       ___decimal_point           1000db24     LIBCMT:nlsdata1.obj
 0003:00000b28       ___decimal_point_length    1000db28     LIBCMT:nlsdata1.obj
 0003:00000b30       __NLG_Destination          1000db30     LIBCMT:exsup.obj
 0003:00000b40       ___abort_behavior          1000db40     LIBCMT:abort.obj
 0003:00000b48       __timezone                 1000db48     LIBCMT:timeset.obj
 0003:00000b4c       __daylight                 1000db4c     LIBCMT:timeset.obj
 0003:00000b50       __dstbias                  1000db50     LIBCMT:timeset.obj
 0003:00000bd8       __tzname                   1000dbd8     LIBCMT:timeset.obj
 0003:00000c00       __lpdays                   1000dc00     LIBCMT:days.obj
 0003:00000c34       __days                     1000dc34     LIBCMT:days.obj
 0003:00000c74       ??_R0?AVbad_exception@std@@@8 1000dc74     LIBCMT:frame.obj
 0003:00000c94       ??_R0?AVexception@std@@@8  1000dc94     LIBCMT:frame.obj
 0003:00000cc4       __aenvptr                  1000dcc4     LIBCMT:dllcrt0.obj
 0003:00000cc8       __wenvptr                  1000dcc8     LIBCMT:dllcrt0.obj
 0003:00000ccc       ___error_mode              1000dccc     LIBCMT:dllcrt0.obj
 0003:00000cd0       ___app_type                1000dcd0     LIBCMT:dllcrt0.obj
 0003:00000ffc       _gpFlsAlloc                1000dffc     LIBCMT:tidtable.obj
 0003:00001000       _gpFlsGetValue             1000e000     LIBCMT:tidtable.obj
 0003:00001004       _gpFlsSetValue             1000e004     LIBCMT:tidtable.obj
 0003:00001008       _gpFlsFree                 1000e008     LIBCMT:tidtable.obj
 0003:00001014       __maxwait                  1000e014     LIBCMT:crtheap.obj
 0003:00001018       __umaskval                 1000e018     LIBCMT:crt0dat.obj
 0003:0000101c       ___argc                    1000e01c     LIBCMT:crt0dat.obj
 0003:00001020       ___argv                    1000e020     LIBCMT:crt0dat.obj
 0003:00001024       ___wargv                   1000e024     LIBCMT:crt0dat.obj
 0003:00001028       __environ                  1000e028     LIBCMT:crt0dat.obj
 0003:0000102c       ___initenv                 1000e02c     LIBCMT:crt0dat.obj
 0003:00001030       __wenviron                 1000e030     LIBCMT:crt0dat.obj
 0003:00001034       ___winitenv                1000e034     LIBCMT:crt0dat.obj
 0003:00001038       __pgmptr                   1000e038     LIBCMT:crt0dat.obj
 0003:0000103c       __wpgmptr                  1000e03c     LIBCMT:crt0dat.obj
 0003:00001040       __exitflag                 1000e040     LIBCMT:crt0dat.obj
 0003:00001044       __C_Termination_Done       1000e044     LIBCMT:crt0dat.obj
 0003:00001048       __C_Exit_Done              1000e048     LIBCMT:crt0dat.obj
 0003:0000115c       __crtheap                  1000e15c     LIBCMT:heapinit.obj
 0003:000012b0       ___sbh_pHeaderDefer        1000e2b0     LIBCMT:sbheap.obj
 0003:000012b4       ___locale_changed          1000e2b4     LIBCMT:setlocal.obj
 0003:000012b8       ___lc_handle               1000e2b8     LIBCMT:nlsdata2.obj
 0003:000012d0       ___lc_codepage             1000e2d0     LIBCMT:nlsdata2.obj
 0003:000012d4       ___lc_collate_cp           1000e2d4     LIBCMT:nlsdata2.obj
 0003:000012dc       ___mbulinfo                1000e2dc     LIBCMT:mbctype.obj
 0003:000012e8       ___mbcodepage              1000e2e8     LIBCMT:mbctype.obj
 0003:000012ec       ___ismbcodepage            1000e2ec     LIBCMT:mbctype.obj
 0003:000012f0       ___mblcid                  1000e2f0     LIBCMT:mbctype.obj
 0003:000012f4       ___pInvalidArgHandler      1000e2f4     LIBCMT:invarg.obj
 0003:0000130c       ?pArgList@UnDecorator@@0PAVReplicator@@A 1000e30c     LIBCMT:undname.obj
 0003:00001310       ?pZNameList@UnDecorator@@0PAVReplicator@@A 1000e310     LIBCMT:undname.obj
 0003:00001314       ?pTemplateArgList@UnDecorator@@0PAVReplicator@@A 1000e314     LIBCMT:undname.obj
 0003:00001318       ?gName@UnDecorator@@0PBDB  1000e318     LIBCMT:undname.obj
 0003:0000131c       ?name@UnDecorator@@0PBDB   1000e31c     LIBCMT:undname.obj
 0003:00001320       ?outputString@UnDecorator@@0PADA 1000e320     LIBCMT:undname.obj
 0003:00001324       ?maxStringLength@UnDecorator@@0HA 1000e324     LIBCMT:undname.obj
 0003:00001328       ?disableFlags@UnDecorator@@0KA 1000e328     LIBCMT:undname.obj
 0003:0000132c       ?m_pGetParameter@UnDecorator@@0P6APADJ@ZA 1000e32c     LIBCMT:undname.obj
 0003:00001330       ?fExplicitTemplateParams@UnDecorator@@0_NA 1000e330     LIBCMT:undname.obj
 0003:00001331       ?fGetTemplateArgumentList@UnDecorator@@0_NA 1000e331     LIBCMT:undname.obj
 0003:0000164c       ?__pInconsistency@@3P6AXXZA 1000e64c     LIBCMT:hooks.obj
 0003:00001670       ___pPurecall               1000e670     LIBCMT:inithelp.obj
 0003:00001678       ?_pnhHeap@@3P6AHI@ZA       1000e678     LIBCMT:handler.obj
 0003:0000167c       ___lconv_static_null       1000e67c     LIBCMT:lconv.obj
 0003:00001688       __newmode                  1000e688     LIBCMT:_newmode.obj
 0003:00001758       ___@@_PchSym_@00@UhhkPhixPhvgUhhkUexlnPkilcbUwooivovzhvUhgwzucOlyq@ 1000e758     stdafx.obj
 0003:00001764       ___sse2_available          1000e764     <common>
 0003:00001768       ___sbh_cntHeaderList       1000e768     <common>
 0003:0000176c       ___sbh_pHeaderList         1000e76c     <common>
 0003:00001770       ___sbh_threshold           1000e770     <common>
 0003:00001774       ___sbh_pHeaderScan         1000e774     <common>
 0003:00001778       ___sbh_sizeHeaderList      1000e778     <common>
 0003:0000177c       ___sbh_indGroupDefer       1000e77c     <common>
 0003:00001780       __debugger_hook_dummy      1000e780     <common>
 0003:00001784       ___active_heap             1000e784     <common>
 0003:00001788       __nhandle                  1000e788     <common>
 0003:000017a0       ___pioinfo                 1000e7a0     <common>
 0003:000018a0       ___env_initialized         1000e8a0     <common>
 0003:000018a4       ___onexitend               1000e8a4     <common>
 0003:000018a8       ___onexitbegin             1000e8a8     <common>
 0003:000018ac       ___mbctype_initialized     1000e8ac     <common>
 0003:000018b0       __FPinit                   1000e8b0     <common>
 0003:000018b4       ___dyn_tls_init_callback   1000e8b4     <common>
 0003:000018b8       __acmdln                   1000e8b8     <common>

 entry point at        0001:000013f7

 Static symbols

 0001:00001062       __onexit_nolock            10002062 f   LIBCMT:onexit.obj
 0001:00001301       ___DllMainCRTStartup       10002301 f   LIBCMT:dllcrt0.obj
 0001:00001ee8       __initterm                 10002ee8 f   LIBCMT:crt0dat.obj
 0001:00001fae       _doexit                    10002fae f   LIBCMT:crt0dat.obj
 0001:000026bc       _parse_cmdline             100036bc f   LIBCMT:stdargv.obj
 0001:00003c90       __updatetlocinfoEx_nolock  10004c90 f   LIBCMT:setlocal.obj
 0001:00003d44       ?CPtoLCID@@YAHH@Z          10004d44 f   LIBCMT:mbctype.obj
 0001:00003d73       ?setSBCS@@YAXPAUthreadmbcinfostruct@@@Z 10004d73 f   LIBCMT:mbctype.obj
 0001:00003dd7       ?setSBUpLow@@YAXPAUthreadmbcinfostruct@@@Z 10004dd7 f   LIBCMT:mbctype.obj
 0001:00004095       ?getSystemCP@@YAHH@Z       10005095 f   LIBCMT:mbctype.obj
 0001:000048b4       __unwind_handler4          100058b4 f   LIBCMT:exsup4.obj
 0001:000050c0       _siglookup                 100060c0 f   LIBCMT:winsig.obj
 0001:00005378       ?x_ismbbtype_l@@YAHPAUlocaleinfo_struct@@IHH@Z 10006378 f   LIBCMT:ismbbyte.obj
 0001:00005f4a       ?__crtGetStringTypeA_stat@@YAHPAUlocaleinfo_struct@@KPBDHPAGHHH@Z 10006f4a f   LIBCMT:a_str.obj
 0001:00006190       ?__crtLCMapStringA_stat@@YAHPAUlocaleinfo_struct@@KKPBDHPADHHH@Z 10007190 f   LIBCMT:a_map.obj
 0001:0000668c       __unwind_handler           1000768c f   LIBCMT:exsup.obj
 0001:00006a77       _fastcopy_I                10007a77 f   LIBCMT:p4_memcpy.obj
 0001:00006be1       _has_osfxsr_set            10007be1 f   LIBCMT:cpu_disp.obj
 0001:00006d0c       _fastzero_I                10007d0c f   LIBCMT:p4_memset.obj
 0001:00006fef       ?strtoxl@@YAKPAUlocaleinfo_struct@@PBDPAPBDHH@Z 10007fef f   LIBCMT:strtol.obj
 0001:00007547       ?CatchGuardHandler@@YA?AW4_EXCEPTION_DISPOSITION@@PAUEHExceptionRecord@@PAUCatchGuardRN@@PAX2@Z 10008547 f   LIBCMT:_trnsctrl_.obj
 0001:00007651       ?TranslatorGuardHandler@@YA?AW4_EXCEPTION_DISPOSITION@@PAUEHExceptionRecord@@PAUTranslatorGuardRN@@PAX2@Z 10008651 f   LIBCMT:_trnsctrl_.obj
 0001:00007a43       ?ExFilterRethrow@@YAHPAU_EXCEPTION_POINTERS@@@Z 10008a43 f   LIBCMT:frame.obj
 0001:00007b06       ?IsInExceptionSpec@@YAEPAUEHExceptionRecord@@PBU_s_ESTypeList@@@Z 10008b06 f   LIBCMT:frame.obj
 0001:00007b81       ?CallUnexpected@@YAXPBU_s_ESTypeList@@@Z 10008b81 f   LIBCMT:frame.obj
 0001:00007bb2       __catch$?CallUnexpected@@YAXPBU_s_ESTypeList@@@Z$0 10008bb2 f   LIBCMT:frame.obj
 0001:00007bca       ?CallCatchBlock@@YAPAXPAUEHExceptionRecord@@PAUEHRegistrationNode@@PAU_CONTEXT@@PBU_s_FuncInfo@@PAXHK@Z 10008bca f   LIBCMT:frame.obj
 0001:00007f77       ?CatchIt@@YAXPAUEHExceptionRecord@@PAUEHRegistrationNode@@PAU_CONTEXT@@PAXPBU_s_FuncInfo@@PBU_s_HandlerType@@PBU_s_CatchableType@@PBU_s_TryBlockMapEntry@@H1E@Z 10008f77 f   LIBCMT:frame.obj
 0001:00007fe5       ?FindHandlerForForeignException@@YAXPAUEHExceptionRecord@@PAUEHRegistrationNode@@PAU_CONTEXT@@PAXPBU_s_FuncInfo@@HH1@Z 10008fe5 f   LIBCMT:frame.obj
 0001:000080d9       ?FindHandler@@YAXPAUEHExceptionRecord@@PAUEHRegistrationNode@@PAU_CONTEXT@@PAXPBU_s_FuncInfo@@EH1@Z 100090d9 f   LIBCMT:frame.obj
 0001:00008710       __unwindfunclet$?InvokeNewDialog@SPVistaCOMProxy@@QAEHW4_NEW_FILE_DIALOG_INVOKE_TYPE@@PAUtagOFNW@@PBU_GUID@@@Z$0 10009710 f    CIL library: CIL module
 0001:0000871b       __unwindfunclet$?InvokeNewDialog@SPVistaCOMProxy@@QAEHW4_NEW_FILE_DIALOG_INVOKE_TYPE@@PAUtagOFNW@@PBU_GUID@@@Z$1 1000971b f    CIL library: CIL module
 0001:00008726       __ehhandler$?InvokeNewDialog@SPVistaCOMProxy@@QAEHW4_NEW_FILE_DIALOG_INVOKE_TYPE@@PAUtagOFNW@@PBU_GUID@@@Z 10009726 f    CIL library: CIL module
 0001:00008750       __unwindfunclet$?AddJumpListSeparator@SPVistaCOMProxy@@AAE_NPAUIObjectCollection@@@Z$0 10009750 f    CIL library: CIL module
 0001:00008758       __unwindfunclet$?AddJumpListSeparator@SPVistaCOMProxy@@AAE_NPAUIObjectCollection@@@Z$1 10009758 f    CIL library: CIL module
 0001:00008760       __ehhandler$?AddJumpListSeparator@SPVistaCOMProxy@@AAE_NPAUIObjectCollection@@@Z 10009760 f    CIL library: CIL module
 0001:00008780       __unwindfunclet$?AddJumpListTask@SPVistaCOMProxy@@AAE_NPAUIObjectCollection@@PB_W1@Z$0 10009780 f    CIL library: CIL module
 0001:00008788       __unwindfunclet$?AddJumpListTask@SPVistaCOMProxy@@AAE_NPAUIObjectCollection@@PB_W1@Z$1 10009788 f    CIL library: CIL module
 0001:00008790       __ehhandler$?AddJumpListTask@SPVistaCOMProxy@@AAE_NPAUIObjectCollection@@PB_W1@Z 10009790 f    CIL library: CIL module
 0001:000087b0       __unwindfunclet$?CreateJumpList@SPVistaCOMProxy@@QAEHPB_W00@Z$0 100097b0 f    CIL library: CIL module
 0001:000087b8       __unwindfunclet$?CreateJumpList@SPVistaCOMProxy@@QAEHPB_W00@Z$1 100097b8 f    CIL library: CIL module
 0001:000087c0       __unwindfunclet$?CreateJumpList@SPVistaCOMProxy@@QAEHPB_W00@Z$2 100097c0 f    CIL library: CIL module
 0001:000087c8       __unwindfunclet$?CreateJumpList@SPVistaCOMProxy@@QAEHPB_W00@Z$3 100097c8 f    CIL library: CIL module
 0001:000087d0       __ehhandler$?CreateJumpList@SPVistaCOMProxy@@QAEHPB_W00@Z 100097d0 f    CIL library: CIL module
 0001:000087eb       __ehhandler$?CallUnexpected@@YAXPBU_s_ESTypeList@@@Z 100097eb f   LIBCMT:frame.obj
 0001:00008810       ??__Fm_proxy@?1??GetProxy@@YAAAVSPVistaCOMProxy@@XZ@YAXXZ 10009810 f    CIL library: CIL module
